:020000000528D1
:0800080009008B010C3084009B
:100010008001840A041F08288316063081000030FE
:100020008500F930860083121F308500FF3086007E
:100030008F211330A5008B01810185210F390838EC
:10004000A30006309D00051208304A210021072137
:100050008614A30B3028CF2085211F390838A30030
:10006000861D36288B18382877203D288D205F285C
:100070008B108610822008304A21A320861D632819
:100080009C1843281021861D6328B920861D6728E7
:100090009C184B281021861D6728AE20861D6B28D2
:1000A0009C1853281021861D6B28C420861D5F28AC
:1000B0009C185B281021861D5F289C012828A320FE
:1000C0009C1863284921C4209C1867284921AE2028
:1000D0009C186B284921B9209C186F2849219D0B39
:1000E0005F2806309D009C0108304A2128281830DE
:1000F0008C0019308D001A308E001B308F000030BC
:100100009C00080014308C0015308D0016308E00D5
:1001100017308F0002309C00080010308C00113026
:100120008D0012308E0013308F0004309C000800C8
:1001300010308C0011308D0012308E0013308F0083
:1001400006309C0008000C08051081000B11061EEB
:10015000AC280B1DA7280B11051408000D088510ED
:1001600081000B11861EB7280B1DB2280B118514B8
:1001700008000E08051181000B11061FC2280B1D77
:10018000BD280B11051508000F08851181000B1102
:10019000861FCD280B1DC8280B11851508000430BB
:1001A000AF000E30850049210D30850049210B300C
:1001B00085004921073085004921AF0BD1280F3038
:0601C0008500060808009E
:100200000030A420010C7F39FF3CAF2008000030F3
:10021000BA20010C7F39FF3CC5200800F5301129B8
:10022000C33081000B1100000B1D1429080032306F
:10023000A00014309F000530A10006152621000003
:100240000000061126219F0B1D29080020089E0092
:100250009E0B2829A10B2F290530A100A00308001F
:100260003230A00014309F000530A10006153F2158
:100270000000000006113F219F0B362908002008CE
:100280009E009E0B4129A10B48290530A100A00A20
:1002900008000301A800861C4F29291050292914A1
:1002A000861001308A00280882076D296B29692988
:1002B00067296529632961295F2975297F29172104
:1002C0000E2117210E2117210E2117210E21172192
:1002D0000E2117210E2117210E2117210E21291879
:1002E0007329861408008610080030210E2117217A
:1002F0000E2130210E2117210E2130216F293021AE
:100300000E2117210E2130216F29A60DA60D261AC8
:10031000013AA61A013AA619013AA60008000C30C3
:100320008400AB011230B0009B218000840AAB0A2C
:10033000B00B942908002B08890083160814831237
:10034000080808002B0889002C08880083168815E7
:0C03500055308900AA308900881408008C
:02400E00F33F7E
:104200002D002D002D002D00870087004B004B0056
:10421000010001000A000A002D002D002D002D00D4
:044220000000060094
:00000001FF
